:100000001AC0FECFFDCFFCCFFBCFFACFF9CFF8CF90
:10001000F7CFF6CFF5CFF4CFF3CFF2CFF1CFF0CFCC
:10002000EFCFEECFEDCFECCFEBCFEACFE9CFE8CFFC
:10003000E7CFE6CF0000F894EE27EFBBE5BFF8E18D
:10004000A895A4B7A77FA4BFF0936000E0936000D9
:100050008DE0A2E0BB27ED938A95E9F780E092E07E
:10006000A0E0B1E0ED930197E9F7E4E3F0E08591DA
:100070009591009761F0A591B59105901590BF01FC
:10008000F00105900D920197E1F7FB01F0CFE0E060
:10009000EEBBE0E0EABDE0E0EBBDEFEFEDBFE2E09C
:1000A000EEBFC0E8D1E04DC0E881E03011F4E0ECF3
:1000B00046C0E13011F4E9EF42C0E23011F4E4EA65
:1000C0003EC0E33011F4E0EB3AC0E43011F4E9E96A
:1000D00036C0E53011F4E2E932C0E63011F4E2E86E
:1000E0002EC0E73011F4E8EF2AC0E83011F4E0E860
:1000F00026C0E93011F4E0E922C0EA3011F4EFEB58
:100100001EC0EB3011F4E6E81AC0EC3011F4EFEA4F
:1001100016C0E1E014C0E881E066E0937C00E09165
:100120007A00E064E0937A00E0917A00E071E1F314
:10013000E0917A00E061E0937A00E0917900219605
:100140000895E0E8E0936100E0E0E0936100EFEF04
:10015000E5B9E4B9E0E0E8B9E7B9EFEFEBB9EAB93E
:10016000E0E0E4BDE5BDE6BDE7BDE8BDE0938000AD
:10017000E0938100E0938500E0938400E0938700A2
:10018000E0938600E0938900E0938800E0938B0081
:10019000E0938A00E093B600E093B000E093B100F2
:1001A000E093B200E093B300E093B400E093690001
:1001B000EDBBE0936800E0936E00E0936F00E09386
:1001C0007000E0E8E0BFE0E0E0937B00ECE3E09368
:1001D0007E00E0E6E0937C00E3E8E0937A00E0E074
:1001E000EA9399DF3E2EE1E0EA9395DF2E2E832CF1
:1001F0009924E22DF0E08E0E9F1E4AD0EAE0F0E056
:100200006ED04F01231418F4E32DE21902C0E22D41
:10021000E3197E2E3FD05DD0E02111F0E4E60AC064
:1002200039D051D0E02111F0662405C0E72D30D03F
:10023000F0E06BD06E2EE4E66E1638F0EBE0EA9359
:1002400033DFE5B9ECE0EA931AC0662039F4EAE05E
:10025000EA932ADFE5B9EAE0EA9311C0A62DEAE0C5
:1002600046D04E2E4A9220DFE5B92F98A42DEAE021
:10027000EA9FF001AE2FE62DEA1B5E2E5A9214DFA4
:10028000EBB9E8ECF0E0FA93EA930CD0A8CFFFCFFB
:10029000D4010895A72DE0E011D00E2EF9DFE0E0A3
:1002A000F0E00895E991F991309639F080ED97E00A
:1002B0000197F1F7A8953197C9F70895EA17E1E09A
:1002C00009F0EE270895EA17FB07E1E009F0EE27B1
:1002D0000895EA17FB07E1E009F4EE270895FA9F75
:1002E000F02DEB9FF00DEA9FE02DF10D0895002415
:1002F00098E0AA0F001C0E1A10F40E0E01C0A160A7
:100300009A95B9F7EA2FA02D08950024112490E1C1
:10031000AA0FBB1F001C111C0E1A1F0A18F40E0E88
:100320001F1E01C0A1609A9599F7FD01D0010895A3
:00000001FF
